:10000000000018308A000E2FFF00030E8301A100AC
:100010000A08A0008A010408A2007708A300780853
:10002000A4007908A5007A08A6007B08A70083131E
:1000300083128C308400801E1F288C1A38288C3044
:100040008400001C25280C183B2822088400230863
:10005000F7002408F8002508F9002608FA00270808
:10006000FB0020088A00210E8300FF0E7F0E09008E
:100070008A110A121F298A110A1298290A108A1055
:100080000A11820731342E34303400340A108A10B9
:100090000A118207683461346E3464346C34653418
:1000A0005F3463346F346D346D345F34723465346F
:1000B0006C34613479340D340A3400340A108A10F7
:1000C0000A11820753346534743420344134643463
:1000D000643472346534733473340D340A34003448
:1000E0000A108A100A11820775347334653420347B
:1000F000453445340D340A3400340A108A100A118C
:1001000082074D34423441345234493420344C3423
:100110006F3461346434203443346F346E34743457
:1001200072346F346C346C34653472342034763409
:1001300031342E3430340D340A3400340A108A102D
:100140000A11820745346E347434653472342034B5
:1001500043346F346D346D3461346E3464340D3433
:100160000A3400340A108A100A11820747344634D0
:1001700030343A3425344C34753400340A108A1043
:100180000A1182074734463431343A3425344C342A
:10019000753400340A108A100A1182074734463435
:1001A00032343A3425344C34753400340A108A1011
:1001B0000A1182074734463433343A3425344C34F8
:1001C0007534003464008C1EE22818088316BE00C3
:1001D00083121A08F8008316BE1CF2288312181224
:1001E0001816831683120034F701F80183160317DB
:1001F000410803104218F707F70CF80CC218F7076C
:10020000F70CF80C4219F707F70CF80CC219F707AE
:10021000F70CF80C421AF707F70CF80CC21AF7079C
:10022000F70CF80C421BF707F70CF80CC21BF7078A
:10023000F70CF80C031383128A110A127E29C030BE
:1002400083164B07840083130317C2010408C100FF
:100250004210831B421483120313E22083160317F8
:100260004108840083134218831778088000C03047
:1002700003134B078400831300082F3C031D5229EE
:10028000FD15CB010317BE013E080A3C031C4F2994
:10029000C0303E07840083138001BE0A44292F30FA
:1002A0000313C000FD1D9329C0304B078400831346
:1002B00000080D3C031D8B294B08043C03188B29B7
:1002C000FD11CB010130BF0041082F3C03188A29E2
:1002D0004108393C031C8A2942082F3C03188A290B
:1002E0004208393C031C8A29303041020317C00000
:1002F000C1000A30C20083120313F4287808831661
:100300000317C100303003134202031741070313E0
:10031000DB008B29BF010130CB074B080B3C0318D6
:100320009329FD11CB0183128C128A110A12252800
:100330002030F8001F08C73978049F001F15F630D9
:100340008F0041308E007E0BA729FE01A9290130C4
:10035000FE00FE08031DAE298710AF2987148316FF
:10036000E2106208870083121F19B4291E08FA00E0
:1003700083161E080317BE007A08BF0083120313FA
:100380006E08831603173F02031CDD29031DD329C2
:100390003E08831203136D02031CD1298316031731
:1003A000DD298316031783120313E7160715831637
:1003B000621162088700E4290317831203130711EF
:1003C000831662116208870083120C108A110A12C8
:1003D00025280C30F7000730810181308400831319
:1003E0000008F0390738800064000008F739F71971
:1003F000F03977048000B53090008A150A16CA2FAC
:10040000031736088D0083168C130C1483120C0806
:10041000F8000313003403173208B20AB500B6001F
:100420000313002278080317B3003208B600031341
:10043000002278080317B4003308F8003408F900E4
:1004400003130034031737088D0038088C00831617
:100450008C130C15831203130B08F7008B138316F0
:10046000031755308D00AA308D008C148C18362A55
:100470000C117708831203138B040034031732081E
:10048000B20AB5003308B6003508B7003308B80023
:100490000313222203173408B5003208B7003408CA
:1004A000B80003132222003420300317CF00CB0101
:1004B000CC01CD01CE014608FA004508F9004408F8
:1004C000F8004308F7000310771C742A4708CB078D
:1004D00048080318480FCC0749080318490FCD07EF
:1004E0004A0803184A0FCE07CE0CCD0CCC0CCB0C0F
:1004F000FA0CF90CF80CF70CCF0B632A0313003439
:10050000F701F801F901FA010317CA01CB01CC0187
:10051000CD0149084804470446040319BF2A203086
:10052000CE000310C20DC30DC40DC50DCA0DCB0DF9
:10053000CC0DCD0D49084D02031DA82A48084C02D8
:10054000031DA82A47084B02031DA82A46084A0291
:10055000031CB92A4608CA024708031C470FCB02EE
:100560004808031C480FCC024908031C490FCD0260
:100570000314F70DF80DF90DFA0DCE0B912A4A3040
:1005800084008317031300340317B501B401031368
:1005900062080317B300031361080317B20035089C
:1005A000C6003408C5003308C4003208C300CA01BD
:1005B000C901C801C830C700031354227A080317C1
:1005C000B6007908B5007808B4007708B30036089B
:1005D000C6003508C5003408C4003308C300CA018A
:1005E000C901C8010530C700031354227A08031754
:1005F000B7007908B6007808B5007708B400B800ED
:1006000040303507B9003608BA001F3003182030D3
:10061000BA073708BB00003003180130BB07BF0121
:100620003B0CBE003A0CBD00390CBC00BE0CBD0C2E
:10063000BC0CBE0CBD0CBC0CBE0CBD0CBC0C0F30FD
:10064000BE053F08C6003E08C5003D08C4003C0882
:10065000C300CA01C9010330C800FF30C70003133B
:1006600054227A080317C0007908BF007808BE003A
:100670007708BD004008C5003F08C4003E08C3001D
:100680003D08C200C901C8010330C700E830C600F8
:10069000031380227808EE007708ED00003403177A
:1006A000B501B401031360080317B30003135F0817
:1006B0000317B2003508C6003408C5003308C4006B
:1006C0003208C300CA01C901C801C830C7000313FA
:1006D00054227A080317B6007908B5007808B400E8
:1006E0007708B3003608C6003508C5003408C400D2
:1006F0003308C300CA01C901C8010530C70003138C
:1007000054227A080317B7007908B6007808B500B4
:100710007708B400B80040303507B9003608BA0091
:100720001F3003182030BA073708BB000030031809
:100730000130BB07BF013B0CBE003A0CBD00390CB9
:10074000BC00BE0CBD0CBC0CBE0CBD0CBC0CBE0C6D
:10075000BD0CBC0C0F30BE053F08C6003E08C500EE
:100760003D08C4003C08C300CA01C9010330C800E9
:10077000FF30C700031354227A080317C00079081A
:10078000BF007808BE007708BD004008C5003F08DC
:10079000C4003E08C3003D08C200C901C8010330BF
:1007A000C700E830C600031380227808F6007708F7
:1007B000F500003494128316E21262088700621674
:1007C00062088700E21562088700253083129400D2
:1007D0000030831694002F308500C0308600193019
:1007E0008700E20083120512831605128312861217
:1007F000831686128312061283160612831286113E
:100800008316861183120611831606118312861031
:100810008316861083120610831606108312871023
:100820008316E21062088700831207118316621193
:1008300062088700831287128316E212620887001B
:1008400083120713831662136208870083128713CB
:100850008316E213620887001F1383121F179F1766
:1008600083169F1783121F1483161F109F101F11CA
:100870009F150730831203178D0083168C130C14F9
:1008800083120C08993C031D602CB20103130B2248
:100890007908E0007808DF0002300317B200031384
:1008A0000B227908E2007808E10004300317B20057
:1008B00003130B227908E4007808E300BE2C031729
:1008C000B201031360080317B40003135F08031792
:1008D000B30003133E2202300317B2000313620871
:1008E0000317B400031361080317B30003133E2278
:1008F00004300317B200031364080317B400031392
:1009000063080317B30003133E220317B201031356
:100910000B227908FA0078085F02031DB12C7A08CF
:100920006002031DB12C02300317B20003130B2227
:100930007908FA0078086102031DB12C7A08620276
:10094000031DB12C04300317B20003130B227908E6
:10095000FA0078086302031DB12C7A0864020319B7
:10096000B32CE714BE2C9930E60007300317B7000C
:10097000031366080317B80003132222C4224F236F
:10098000C0308B0483160C130C1483126C1FC92CFB
:100990006C158A150A12BD294D3084008317000892
:1009A0000319E32C0130F800BF30F7006400F70BA7
:1009B000D62CF80BD42C4A30F700F70BDD2C0000B6
:1009C0006400800BD22C00341F151F19E52C1E0863
:1009D000FA0083161E08F1007A08F200F301F40110
:1009E000740883120317C6007308C5007208C40098
:1009F0007108C300CA01C9010330C800E830C7004C
:100A0000031354227A080317C1007908C00078083C
:100A1000BF007708BE004108C5004008C4003F0879
:100A2000C3003E08C200C901C8010330C700FF303F
:100A3000C600031380227A080317C2007908C10098
:100A40007808C0007708BF004208C6004108C5000A
:100A50004008C4003F08C300CA01C9013708C800E4
:100A60003608C700031354227A08F4007908F3000B
:100A70007808F2007708F1000317C101C0013508BA
:100A8000BF003408BE004108C6004008C500350854
:100A9000C4003408C300CA01C9010330C800E830EB
:100AA000C700031354227A080317C2007908C10053
:100AB0007808C0007708BF000310420CFA00410C10
:100AC000F900400CF8003F0CF700F1027808031C15
:100AD000780FF2027908031C790FF3027A08031CDD
:100AE0007A0FF4027408C5007308C4007208C300CA
:100AF0007108C200C901C801C7013908C600031343
:100B000080227A08F4007908F3007808F200770868
:100B1000F10074080317C5007308C4007208C3000D
:100B20007108C200C901C801C7013808C600031313
:100B300080227A08F4007908F3007808F200770838
:100B4000F100003483166008840083136118831752
:100B5000831203174A088000840A80018316031356
:100B6000E00A0319E10A8312003404080317B700EE
:100B70003B30BE009A30BD00CA30BC00BB010A3019
:100B8000B9003608C5003508C4003408C30033086E
:100B9000C2003E08C9003D08C8003C08C7003B0829
:100BA000C6000313802200080317B300840A00085C
:100BB000B400840A0008B500840A0008B600F708EB
:100BC000031DF52D3908013A0319F52D37080319CE
:100BD000F62D0F3939020319EF2D0318FD2DB71B20
:100BE000FD2D371BF62D2030F72DB7013030F707DC
:100BF0007708CA000313A22503173E08C5003D0865
:100C0000C4003C08C3003B08C200C901C801C701B9
:100C10000A30C600031380227A080317BE00790841
:100C2000BD007808BC007708BB00B90BC12D0313C9
:100C300000340317B4013308FA0032088400831328
:100C40007A18831780080319422E34080A3C031CC3
:100C5000422E3308FA003208B20A0319B30A84009C
:100C600083137A1883170008B500031313080317BA
:100C70003508031393008316141C3C2E83120317AC
:100C8000B40A1B2E031300341F151F19452E1E080E
:100C9000FA0083161E08F1007A08F200F301F4014D
:100CA000740883120317C6007308C5007208C400D5
:100CB0007108C300CA01C9010330C800E830C70089
:100CC000031354227A080317B6007908B500780890
:100CD000B4007708B3003608C5003508C4003408EE
:100CE000C3003308C200C901C8010330C700FF3088
:100CF000C600031380227A080317B7007908B600EC
:100D00007808B5007708B4003208F700F801F90157
:100D1000FA017A08BB007908BA007808B9003208ED
:100D2000B8003708C6003608C5003508C4003408C6
:100D3000C3003B08CA003A08C9003908C800320895
:100D4000C700031354227A08F4007908F3007808E6
:100D5000F2007708F100003404080317B7003B30B5
:100D6000BE009A30BD00CA30BC00BB010A30B900D9
:100D70003608031DB7033508C5003408C40033081E
:100D8000C3003208C2003E08C9003D08C8003C0844
:100D9000C7003B08C6000313802200080317B200F7
:100DA000840A0008B300840A0008B400840A00081A
:100DB000B500FD308407F708031DF12E360A39020D
:100DC0000319F12E37080319F22E0F3939020319CE
:100DD000EB2E0318092FB71B092F371BF22E2030DB
:100DE000032FB70136083902031D022F7708B70019
:100DF0002E30CA000313A22503173708F70020304E
:100E0000B70500303030F7077708CA000313A22572
:100E100003173E08C5003D08C4003C08C3003B085A
:100E2000C200C901C801C7010A30C60003138022ED
:100E30007A080317BE007908BD007808BC0077085F
:100E4000BB00B90BBB2E031300340317B401831688
:100E50000313141C292F831203173408320784004C
:100E6000831333188317031313088000003A031900
:100E7000482F031734080A3C0318402F0313482F48
:100E8000B40A64001030F700F70B442F2D2F031322
:100E900000340317BA010408B9003A10831B3A144E
:100EA000330EF038B500B507E23EB600323EB8006A
:100EB00033080F39B607B607B807E93EB700B707DA
:100EC000B707320E0F39B707B807B70DB80DB80915
:100ED000B80D32080F39B807B50D0730B4000A3025
:100EE000B807B703031C702FB707B603031C742F92
:100EF000B607B503031C782FB507B403031C7C2F7A
:100F000034308400831707303905391384073830AB
:100F10000402031939170008F700031D972F391B26
:100F2000972F391AAB2FB919972F20309A2FB9154F
:100F300039123030F707B3010408B2003310831BB5
:100F400033147708CA000313A2250317320884005C
:100F5000831333188317840A391F872F0313003430
:100F600003174908F80148020318B92F4808F70089
:100F7000C52FF7010830CA00C80DF70D49087702E0
:100F80000318F700F80DCA0BBC2F03130034031726
:100F9000C91BDC2F0F30F700480EF7050A30770227
:100FA0000318D52F3030F707D72F4908F7077708F0
:100FB000CA000313A22503170F30C8050A304802E0
:100FC0000318E42F3030E62FC9134908C807480832
:100FD000CA000313A22500340317C6080319F92F0A
:100FE0000313E7106711E7116712E71267136C111B
:0E0FF00003170313E7136C10EC10EC11003420
:101000000317BA01B8010A30B900B701B601B5013A
:10101000B40132083304031D1228F701F801F90165
:10102000FA016C293A08BA0A32078400831333188C
:1010300083170008BB003B082D3C031D2B28013003
:10104000B8003A08BA0A32078400831333188317AA
:101050000008BB0038283B082B3C031D38283A0801
:10106000BA0A320784008313331883170008BB00C1
:101070003B082F3C031853293B08393C031C5329D8
:101080003B08303C031D64283A0832078400831370
:10109000331883170008783C031958283A08320798
:1010A00084008313331883170008583C031D6428F9
:1010B0001030B900BA0A3A08BA0A3207840083131A
:1010C000331883170008BB0039080A3C031DBA28EF
:1010D0003B082F3C0318B9283B08393C031CB928AE
:1010E0000310340DBD00350DBE00360DBF00370DA9
:1010F000C000340DF700350DF800360DF900370D3E
:10110000FA00F70DF80DF90DFA0DF70DF80DF90DC0
:10111000FA0DF830F70577083D07B4003E08B50032
:1011200078080318780FB5073F08B6007908031848
:10113000790FB6074008B7007A0803187A0FB70787
:1011400030303B02B407003003180130B5070030DF
:1011500003180130B607003003180130B7073A080A
:10116000BA0A320784008313331883170008BB00C0
:10117000682853293908103C031D53293B08603C5B
:101180000318C9283B087A3C031CC9283B08DF39EF
:10119000CA283B08BB003B082F3C0318D3283B0858
:1011A000393C0318DB283B08403C031853293B0813
:1011B000463C031C53293B082F3C031810293B08CD
:1011C000393C031C1029340DBD00350DBE00360D11
:1011D000BF00370DC000BD0DBE0DBF0DC00DBD0D54
:1011E000BE0DBF0DC00DBD0DBE0DBF0DC00DF0304D
:1011F000BD0530303B023D07B4003E08B50000306D
:1012000003180130B5073F08B6000030031801305D
:10121000B6074008B700003003180130B7073D2972
:10122000340DBD00350DBE00360DBF00370DC000BA
:10123000BD0DBE0DBF0DC00DBD0DBE0DBF0DC00D52
:10124000BD0DBE0DBF0DC00DF030BD0541303B02E0
:101250000A3E3D07B4003E08B500003003180130D7
:10126000B5073F08B600003003180130B607400844
:10127000B700003003180130B7073A08BA0A32073E
:1012800084008313331883170008BB00603C0318E5
:1012900050293B087A3C031C50293B08DF3951296F
:1012A0003B08BB00CB2839080A3C031D6429380BD6
:1012B0006429B409B509B609B709B40A0319B50A0E
:1012C0000319B60A0319B70A3408F7003508F800FD
:1012D0003608F9003708FA000313003478080317BA
:1012E0004608C8006430C9008A110313B0278A1564
:1012F00077080317C60078083030031D8629C71CFD
:101300009129C7199129471A20308929C7114712F5
:101310004714F8077808CA008A110313A2258A1512
:1013200003174608C8000A30C9008A110313B02702
:101330008A1577080317C60078083030031DA629E0
:10134000C719AE29471CAE29471A2030F80778087C
:10135000CA008A110313A2258A1503173030C60765
:101360004608CA008A110313A2258A1500341C30CE
:1013700003179B008A110313DA2B8A15871483162F
:10138000E210620887006400141CB22D8312130857
:1013900003179B001B0B272A0830F80003131F08B4
:1013A000C73978049F008614831686100130831293
:1013B0000317CD008A110313CC248A1501300317BB
:1013C000B3008130B2001030B500B4013308B7006B
:1013D0003208B6008730B8000530B9008A1103130F
:1013E000E4248A158610831686100130E1001C3033
:1013F000E00083120317B20132088A110313B220EE
:101400008A150317B20AF700CA008A110313A2252E
:101410008A15043003173202031DFC294130840071
:101420007408B6007308B5007208B4007108B30000
:101430008A110313B5258A1501300317B3001C3038
:10144000B2008A11031319268A15AF2D03171B0842
:10145000023C031D862A0830F80003131F08C73911
:1014600078049F00061583160611013083120317B6
:10147000CD008A110313CC248A1501300317B30061
:101480008130B2001030B500B4013308B700320823
:10149000B6008730B8000530B9008A110313E42480
:1014A0008A150611831606110130E1001C30E00098
:1014B00083120317B20132088A110313BE208A1562
:1014C0000317B20AF700CA008A110313A2258A156E
:1014D000043003173202031D5B2A41308400740874
:1014E000B6007308B5007208B4007108B3008A1121
:1014F0000313B5258A1501300317B3001C30B20061
:101500008A11031319268A15AF2D03171B08033CF4
:10151000031DE52A0830F80003131F08C7397804B3
:101520009F00861583168611013083120317CD00A4
:101530008A110313CC248A1501300317B3008130BC
:10154000B2001030B500B4013308B7003208B6005D
:101550008730B8000530B9008A110313E4248A15D6
:101560008611831686110130E1001C30E0008312E1
:101570000317B20132088A110313CA208A15031710
:10158000B20AF700CA008A110313A2258A15043093
:1015900003173202031DBA2A413084007408B600D2
:1015A0007308B5007208B4007108B3008A11031300
:1015B000B5258A1501300317B3001C30B2008A111B
:1015C000031319268A15AF2D03171B08043C031DAE
:1015D000442B0830F80003131F08C73978049F0014
:1015E000061683160612013083120317CD008A11E6
:1015F0000313CC248A1501300317B3008130B200E5
:101600001030B500B4013308B7003208B600873097
:10161000B8000530B9008A110313E4248A150612B4
:10162000831606120130E1001C30E000831203171C
:10163000B20132088A110313D6208A150317B20AA1
:10164000F700CA008A110313A2258A150430031774
:101650003202031D192B413084007408B600730850
:10166000B5007208B4007108B3008A110313B525E0
:101670008A1501300317B3001C30B2008A1103131E
:1016800019268A15AF2D03171B08323C031D782B32
:101690000030F80003131F08C73978049F000C308E
:1016A0000317B2008A11031344268A1501308316EA
:1016B000E1001C30E0000530840074088312031739
:1016C000B5007308B4007208B3007108B2000330AB
:1016D000B6008A110313AC268A1501300317B30034
:1016E0001C30B2008A11031319268A15AF2D031777
:1016F0001B08333C031DB32B2030F80003131F08D5
:10170000C73978049F0010300317B500B401B70043
:10171000B601C830B8000530B9008A110313E424BB
:101720008A1501308316E1001C30E000053084008A
:10173000740883120317B5007308B4007208B3006D
:101740007108B2000330B6008A110313AC268A1563
:1017500001300317B3001C30B2008A11031319269D
:101760008A15AF2D03171B083C3C031D0A2C0130C2
:10177000B3002730B2008A11031325278A150130E0
:101780000317B3002730B200031300207808E000ED
:101790007708DF0001308316E1001C30E0001030D4
:1017A0008400831260080317B30003135F08031754
:1017B000B2008A11031349278A1501300317B300B9
:1017C0001C30B2008A11031319268A158A114F237F
:1017D0008A150317B201031360080317B40003133B
:1017E0005F080317B3008A1103133E228A150317FB
:1017F000B2018A1103130B228A157908FA007808BE
:101800005F02031D072C7A0860020319082CE714F5
:10181000AF2D03171B083D3C031D632C0130B300A3
:101820002730B2008A11031325278A1501300317C8
:10183000B3002730B200031300207808E2007708D5
:10184000E10001308316E1001C30E000103084001C
:10185000831262080317B300031361080317B20071
:101860008A11031349278A1501300317B3001C306E
:10187000B2008A11031319268A158A11C4228A1507
:1018800002300317B200031362080317B4000313F6
:1018900061080317B3008A1103133E228A15023030
:1018A0000317B2008A1103130B228A157908FA0074
:1018B00078086102031D602C7A0862020319612C0A
:1018C000E714AF2D03171B083E3C031DB92C013054
:1018D000B3002730B2008A11031325278A1501307F
:1018E0000317B3002730B200031300207808E40088
:1018F0007708E30001308316E1001C30E00010306F
:101900008400831264080317B300031363080317EA
:10191000B2008A11031349278A1501300317B30057
:101920001C30B2008A11031319268A1504300317DC
:10193000B200031364080317B4000313630803170A
:10194000B3008A1103133E228A1504300317B20034
:101950008A1103130B228A157908FA0078086302AA
:10196000031DB62C7A0864020319B72CE714AF2DB7
:1019700003171B08463C031DD82C0313861283163D
:1019800086120130E1001C30E000831203171B08AF
:10199000C6001B30C70003136E2101300317B300CC
:1019A0001C30B2008A11031319268A15AF2D0317B4
:1019B0001B08473C031DF72C03138616831686125B
:1019C0000130E1001C30E000831203171B08C60041
:1019D0001B30C70003136E2101300317B3001C3006
:1019E000B2008A11031319268A15AF2D03171B089D
:1019F000503C031D8F2D003003136719013003176E
:101A0000B30100300313E71901300030031733042A
:101A1000B50000300313671A0130F700770CF701A7
:101A20000318F717770803173504B70000300313BE
:101A3000E71A0130F700F70EF70DF70DC030F70584
:101A4000770803173704B90000300313671B013010
:101A5000F700F70EF70DE030F705770803173904A4
:101A6000BB0000300313E71B0130F700F70EF03026
:101A7000F705770803173B04BD00003003136C180B
:101A80000130F700F70DF70DF70DF830F70577087F
:101A900003173D04BF0000300313EC180130F700BA
:101AA000F70DF70DFC30F705770803173F04C10069
:101AB000003003136C190130F7000310F70D77089D
:101AC00003174104C30000300313EC19013003175E
:101AD00043040313E800E90101308316E1001C30E0
:101AE000E000831269080317C8003730C9008A1163
:101AF0000313C7278A1568080317C8003730C900C1
:101B00008A110313C7278A1501300317B3001C304D
:101B1000B2008A11031319268A15AF2D03171B086B
:101B2000513C031DB02D0130C6008A110313EC2770
:101B30008A1501308316E1001C30E0008312031780
:101B40001B08C6001B30C70003136E2101300317AA
:101B5000B3001C30B2008A11031319268A1503172B
:101B600083160313C32983128A150A16D62F8C1ED7
:101B7000BD2D8A11E2208A15B72D83168612831295
:101B800086120034B7258316BF018C16C03083122D
:101B90008B048A110A164028831686128312861631
:101BA0000034CC250317C801C7014808013C031CB9
:101BB000F92D031DDF2D4708903C031CF92D8316DA
:101BC0000313E217620887008312871BEC2D0317AB
:101BD000C801C701F22D031364001030F700F70BA2
:101BE000EF2D0317C608031D6400C70A0319C80AAE
:101BF000D52D0313B72500340C1EFC2D03174E08FA
:101C0000031399008A150A12252E03174C1003138B
:101C1000CC250317C9014908043C031C472E831631
:101C200003133E1383120317CA0146084A0203181E
:101C30002B2E4808FA00470884008313481883179E
:101C40000008CD00CE000313FC2D0317C70A0319AB
:101C5000C80ACA0A152E831603133E1B3C2E831294
:101C60006F080317CD008A110313CC248A150317BC
:101C70004C14472E8316031383126F080317CD00ED
:101C80008A110313CC248A150317C90A0B2E0313D8
:101C9000B725003003174C180130F8000313003447
:101CA00003179D011D081B07840083131C1883174D
:101CB000800803195D2E9D0A522EC6010313D125FB
:101CC00003171D08C6001C08C8001B08C700031323
:101CD0000526F808031D742E0A300317CD008A115B
:101CE0000313CC248A15602E003403179B080319B4
:101CF000842E83160313BF080319812E8312031742
:101D0000842E8312752E031783160313BF08031D39
:101D10008D2E0030F800482F482F83126508831657
:101D20005B02031D442F43083F3C031DE02E440883
:101D3000403C03189F2E44085A3C0318A72E440821
:101D4000603C0318E02E44087A3C031CE02EE101BD
:101D5000CC30E000430883120317CA008A11031332
:101D6000A2258A158316440883120317CA008A1114
:101D70000313A2258A1583164408673C031DDA2E37
:101D8000E101D030E000450883120317CA008A1130
:101D90000313A2258A150317B301D030B200031331
:101DA00000207A088316DF007908DE007808DD005D
:101DB0007708DC00BF017D170130F800482F432F62
:101DC0004308403C0318E82E43085A3C0318F02E01
:101DD0004308603C0318402F43087A3C031C402F03
:101DE000E101CC30E000430883120317CA008A11D6
:101DF0000313A2258A158316E101D030E0004408C0
:101E000083120317CA008A110313A2258A158316A9
:101E1000450883120317CA008A110313A2258A15E5
:101E20008316460883120317CA008A110313A225DA
:101E30008A158316470883120317CA008A110313F1
:101E4000A2258A158316480883120317CA008A112F
:101E50000313A2258A150317B301D030B200031370
:101E600000207A088316DF007908DE007808DD009C
:101E70007708DC00BF017D130130F800482F432FA5
:101E80000030F800482F482FBF010030F800482FDD
:101E900083128A150A16CE2D03171C08FA001B0898
:101EA000840083137A18831700089F001E08FA0025
:101EB0001D08840083137A18831700081F02031D6E
:101EC000782F1C08FA001B08840083137A188317E4
:101ED0008008031D6E2F0030F800912F1C08FA00B7
:101EE0001B089B0A03199C0A9D0A03199E0A4D2F81
:101EF0001C08FA001B08840083131C1883170008B1
:101F00009F001E08FA001D08840083131E18831703
:101F100000081F0203188F2FFF30FA00902F0130A6
:101F2000F800031300347D18A12F0616831606123D
:101F30007D14553083120317CD008A110313CC246E
:101F40008A1500340317C801480846078400831324
:101F5000471883170313130893018316141CAE2F1D
:101F6000831213088000003A0319C52F031748088D
:101F70000A3C0318BD2F0313C52FC80A6400A630FE
:101F8000F700F70BC12FA42F03130034FD18CD2F3A
:101F90000612831606127D1083120034831603176F
:101FA0003808BA003708BC003608BB003908003CC6
:101FB0000318EF2F3C08FA003B08840083137A18BB
:101FC00083173A080002031DEA2F3B08F8003C087B
:101FD000F900F22FBB0A0319BC0AB903D62F00304F
:101FE000F800F900831203130034F52F8A150A163E
:021FF000DB2FE5
:102000000F3083168500C130860093308700E200D0
:102010008312051283160512831285128316851208
:1020200083128610831686108312061183160611FA
:1020300083128611831686118312061283160612E6
:102040008312861283168612831207118316621179
:1020500062088700831287118316E21162088700E5
:10206000831287128316E212620887008312071315
:1020700083166213620887000A128A158312C22D22
:102080000A168A1194128316E212620887006216F9
:1020900062088700E21162088700213083129400F1
:1020A0000030831694001F1383121F179F17831687
:1020B0009F1783121F1483161F149F101F159F153F
:1020C0000730831203178D0083168C130C148312B0
:1020D0000C08993C031DCA28B2010A1203130B22F3
:1020E0000A167908E0007808DF0002300317B20012
:1020F0000A1203130B220A167908E2007808E1009D
:1021000004300317B2000A1203130B220A167908CF
:10211000E4007808E300053003178D0083168C1364
:102120000C1483120C080313E500063003178D000E
:1021300083168C130C1483120C08F8000C18A428B6
:1021400003136710A6280317031367148316E1010E
:10215000A030E000831203179B011B080A1203132F
:1021600070200A1603179B0AF700CA000A1203130D
:10217000A2250A16083003171B02031DAD289C0177
:10218000A0309B000A128A15031350260A168A11E2
:102190006E290317B201031360080317B400031379
:1021A0005F080317B3000A1203133E220A16023017
:1021B0000317B200031362080317B4000313610886
:1021C0000317B3000A1203133E220A160430031742
:1021D000B200031364080317B40003136308031762
:1021E000B3000A1203133E220A1605300317B20089
:1021F000B401031365080317B3000A1203133E2248
:102200000A1600306718013003179B000630B20031
:10221000B4011B08B3000A1203133E220A16031767
:10222000B2010A1203130B220A167908FA00780881
:102230005F02031D5D297A086002031D5D290230DB
:102240000317B2000A1203130B220A167908FA00C8
:1022500078086102031D5D297A086202031D5D2969
:1022600004300317B2000A1203130B220A1679086E
:10227000FA0078086302031D5D297A086402031DD1
:102280005D29053003178D0083168C130C148312FF
:102290000C0803136502031D5D2900306718013027
:1022A00003179B0006308D0083168C130C148312C9
:1022B0000C081B0203196029031367156E29031705
:1022C00099300313E60007300317B70003136608BD
:1022D0000317B8000A12031322220A16671C80296A
:1022E000061583160611083083120317CD000A1253
:1022F0000313CC240A160611831606118E298312A5
:10230000861483168610083083120317CD000A1234
:102310000313CC240A1686108316861083126C1FB2
:10232000D7296C158316E101A030E0008312031752
:102330009B011B080A1203137D200A1603179B0A30
:10234000F700CA000A120313A2250A161C3003174D
:102350001B02031D99299C01A0309B000A128A15BB
:10236000031350260A168A118316E101A030E000FB
:10237000831203179B011B080A1203139E200A16DF
:1023800003179B0AF700CA000A120313A2250A16B4
:102390000F3003171B02031DBB299C01A0309B00BB
:1023A0000A128A15031350260A168A111B2A83164D
:1023B000E101A030E000831203179B011B080A1201
:1023C00003137D200A1603179B0AF700CA000A129E
:1023D0000313A2250A161C3003171B02031DDE2956
:1023E0009C01A0309B000A128A15031350260A167E
:1023F0008A118316E101A030E000831203179B01CC
:102400001B080A1203139E200A1603179B0AF700E3
:10241000CA000A120313A2250A160F3003171B0263
:10242000031D002A9C01A0309B000A128A15031389
:1024300050260A168A118A150A16C72D10308316DF
:102440000317BA00F701FA01B70CB60C031C2E2AC9
:102450003808F7070318FA0A3908FA07FA0CF70CD4
:10246000F90CF80CBA0B242A031383128A110A16EA
:10247000A72C0030E71801300317C7010030031301
:1024800067190130003003174704C90000300313F7
:10249000E7190130003003174904CB000030031363
:1024A000671A0130F700770CF7010318F717770860
:1024B00003174B04CD0000300313E71A0130F70077
:1024C000F70EF70DF70DC030F705770803174D0429
:1024D000CF0000300313671B0130F700F70EF70D34
:1024E000E030F705770803174F04D10000300313DD
:1024F000E71B0130F700F70EF030F70577080317F8
:102500005104D300003003136C180130F700F70DAD
:10251000F70DF70DF830F705770803175304D500CA
:1025200000300313EC180130F700F70DF70DFC3005
:10253000F705770803175504D700003003136C190B
:102540000130F7000310F70D770803175704D9007F
:1025500000300313EC190130031759040313E8008A
:10256000E9017D1C242D1308503093008316141CA0
:10257000B72A323083120317CD000A120313CC247A
:102580000A160317C701E330C6000A128A1503139F
:10259000A2270A168A110317C701E330C6004708AD
:1025A000C9004608C8004908FA0048088400831397
:1025B0007A18831780080319E12AC80A0319C90A7F
:1025C000D32A46084802F7004908FA004708031CC6
:1025D000470FFA027708F8007A08F9007908C7006F
:1025E0007808C600C708031DF92A4608033C0318EB
:1025F0001F2DC701E330C600C901C8011030CA0051
:10260000D101D20130308316900031309100323048
:1026100092003330930034309400353095003630DA
:102620009600373097003830980039309900613083
:102630009A0062309B0063309C0064309D006530DE
:102640009E0066309F006730A0006830A1006930AE
:10265000A2006A30A3006B30A4006C30A5006D307E
:10266000A6006E30A7006F30A8007030A90071304E
:10267000AA007330AB007430AC007530AD0076301A
:10268000AE007730AF007830B0007930B1007A30EA
:10269000B200B30183124708CC004608CB004C08B7
:1026A000FA004B08840083137A1883170008203C33
:1026B000031D5E2BCB0A0319CC0A4F2B4C08FA00E2
:1026C0004B08840083134C18831700082D3C031912
:1026D000742B4C08FA004B08840083134C188317A2
:1026E00000082B3C031D802B4C08FA004B08CB0A3A
:1026F0000319CC0A840083137A1883170008812BEE
:102700002B30D30053082D3C031D952B480849045A
:102710000319912B4808840083134918831746082E
:1027200080000030F800F900182DCA1BA02B4A0BBE
:102730009A2BA02BCA1BB02B4A08243C0318B02BA1
:10274000480849040319AB2B48088400831349182F
:102750008317460880000030F800F900182D462C39
:10276000CA0803190B2C4A08103C031DDA2B4C082D
:10277000FA004B08840083137A1883170008303C52
:10278000031DDA2B01304B07840083134C18831789
:102790000008783C0319D62B01304B0784008313C3
:1027A0004C1883170008583C031DDA2B0230CB0766
:1027B0000318CC0A4A08083C031DED2B4C08FA000C
:1027C0004B08840083137A1883170008303C031DDC
:1027D000ED2B0130CB070318CC0A4A08023C031D3D
:1027E0000A2C4C08FA004B08840083137A188317CC
:1027F0000008303C031D0A2C01304B078400831372
:102800004C1883170008623C031D0A2C0230CB07CA
:102810000318CC0A462C4C08FA004B08840083139A
:102820007A1883170008303C0319192C0A30CA00A3
:10283000462C01304B07840083134C188317000883
:10284000783C03192D2C01304B07840083134C185E
:1028500083170008583C031D342C1030CA00023086
:10286000CB070318CC0A462C01304B078400831396
:102870004C1883170008623C031D442C0230CA0028
:10288000CB070318CC0A462C0830CA004C08CE00EF
:102890004B08CD004C08FA004B08840083137A18CB
:1028A00083170008303C031D592CCB0A0319CC0AAE
:1028B0004A2C4C08FA004B08840083134C188317E9
:1028C0000008D400403C03186C2C54085A3C031CEC
:1028D0006C2C540820386D2C5408D5000130831618
:1028E000B7009030B600831254088316B8008312E4
:1028F0004A088316B9000A128A1583120313CE27D9
:102900000A168A1179080317D0007808CF00CF087B
:10291000031D8D2CD0080319F22CFA014A08F70088
:10292000CA1BFA03D4007A08D50052088316B700F0
:10293000831251088316B600831255088316B90016
:10294000831254088316B800831203131E2A7908D1
:102950000317D6007808D50090304F02F7005008D2
:10296000FA000130031C0230FA0277085507F8001C
:1029700056080318560FFA077808D1007A08D200D3
:10298000CB0A0319CC0A4C08FA004B0884008313C5
:102990004C1883170008D400403C0318D62C540868
:1029A0005A3C031CD62C54082038D72C5408D50088
:1029B00001308316B7009030B60083125408831696
:1029C000B80083124A088316B9000A128A158312C6
:1029D0000313CE270A168A1179080317D000780846
:1029E000CF00872C4B084D02031D092D4C084E02C9
:1029F000031D092D480849040319052D48088400C2
:102A0000831349188317460880000030F800F90046
:102A1000182D480849040319142D4808840083130D
:102A2000491883174B0880005108F8005208F90034
:102A300079080313EB007808EA001E2D031703132F
:102A40006A08E8046B08E90401308316E1001E30CF
:102A5000E0002A3083120317CA000A120313A225CA
:102A60000A1665080317C6000130C7000A128A1546
:102A700003136E210A168A1103171B08840083139F
:102A80001C1883170030000403195A2DC7010408CD
:102A9000C6004710831B47140008CA000A1203131C
:102AA000A2250A16031746088400831347188317C4
:102AB000840A422D031369080317C8003730C90080
:102AC0000A120313C7270A1668080317C80037300D
:102AD000C9000A120313C7270A160D300317CA00CC
:102AE0000A120313A2250A160A300317CA000A1293
:102AF0000313A2250A1603179D011E301D0784002B
:102B0000831780080319862D9D0A7D2DC6010A12A0
:102B10008A150313D1250A168A1103171D08C6004A
:102B20000130C8001E30C7000A128A15031305269B
:102B30000A168A11F808031DA52D0A300317CD00C7
:102B40000A120313CC240A168D2D0317C6010A128C
:102B50000313EC270A1600348316DC08031D032E2A
:102B6000DD08031D032EDE08031D032EDF08031DF1
:102B7000032E0A128A15831293270A168A11130844
:102B8000463093008316141CC32D32308312031772
:102B9000CD000A120313CC240A160317C701E33031
:102BA000C6000A128A150313A2270A168A110317F0
:102BB000B301E330B2000A128A15031300200A168B
:102BC0008A117A0803179E0079089D0078089C00F6
:102BD00077089B00463C031DF62D9C08031DF62D2F
:102BE0009D08031DF62D9E080319FA2D0313EC15FD
:102BF000012E0317FD100A128A150313C6270A16A1
:102C00008A115C2E83165C0B5A2EDD08031D5A2E8A
:102C1000DE08031D5A2EDF08031D5A2E83120616E6
:102C2000831606127D14553083120317CD000A1245
:102C30000313CC240A161308473093008316141C80
:102C40001F2E323083120317CD000A120313CC2437
:102C50000A160317C701E330C6000A128A150313C8
:102C6000A2270A168A110317B301E330B2000A1231
:102C70008A15031300200A168A117A0803179E008A
:102C800079089D0078089C0077089B00473C031D4D
:102C9000522E9C08031D522E9D08031D522E9E0885
:102CA0000319562E0313EC15582E0317FD140313A6
:102CB0005C2E831683126C1403179C019B01031373
:102CC00039228A150A16E32D8316E101A030E000AF
:102CD000831203179B011B080A12031346200A16CE
:102CE00003179B0AF700CA000A120313A2250A164B
:102CF000133003171B02031D6B2E9C01A0309B0099
:102D00000A128A15031350260A168A118316DC0844
:102D1000031DA62EDD08031DA62EDE08031DA62E0C
:102D2000DF08031DA62E8312861483168610083032
:102D300083120317CD000A120313CC240A1686103F
:102D40008316861083126710C62E83165C0BC42E62
:102D5000DD08031DC42EDE08031DC42EDF08031D7D
:102D6000C42E83120615831606110830831203172A
:102D7000CD000A120313CC240A160611831606117D
:102D800083126714C62E831683126C1400306718E2
:102D9000013003179B000630B200B4011B08B300DA
:102DA0000A1203133E220A16003067180130031777
:102DB0009B000630B2000A1203130B220A16790890
:102DC000FA00780803171B02031DE92EFA080319FD
:102DD000EC2E0313671503179C019B010313392283
:102DE0008A150A16F52D8316DC08031D022FDD084F
:102DF000031D022FDE08031D022FDF08031D022F13
:102E00007D11122F5C0B0F2FDD08031D0F2FDE0825
:102E1000031D0F2FDF08031D0F2F7D15122F8312A7
:102E20006C148316831203179C019B010313392230
:102E30008A150A16072E0715831662116208870085
:102E40000030F80083121F08C73978049F0009304A
:102E50000317CD000A120313CC240A1619300317E6
:102E6000B2000A12031344260A16071183166211D0
:102E700062088700E101A030E0000530840074089A
:102E800083120317B5007308B4007208B300710809
:102E9000B2000330B6000A120313AC260A16031759
:102EA0009C01A0309B00031339228A150A16192EA3
:102EB0000A128A1593270A168A11130832309300D2
:102EC0008316141C612F323083120317CD000A12AF
:102ED0000313CC240A160317C701E330C6000A12F5
:102EE0008A150313A2270A168A110A128A15C62701
:102EF0000A168A118316E101A030E000E330840055
:102F000083130030000403199D2F831203179C01C3
:102F100004089B001C10831B1C140008CA000A1222
:102F20000313A2250A1603171B08840083131C1819
:102F30008317840A83160313812F831203179C01BE
:102F4000A0309B00031339228A150A162B2E071571
:102F500083166211620887000830F80083121F0888
:102F6000C73978049F0009300317CD000A120313F4
:102F7000CC240A1610300317B500B401B700B6010F
:102F8000C830B8000530B9000A120313E4240A1649
:102F900007118316621162088700E101A030E0008A
:102FA00005308400740883120317B5007308B40059
:102FB0007208B3007108B2000330B6000A1203139E
:102FC000AC260A1603179C01A0309B00031339227C
:102FD0008A150A163D2E03179C019B010313392203
:062FE0008A150A16AF2E4F
:103000000A1293270A161308333093008316141CF0
:103010000728323083120317CD000A128A110313D6
:10302000CC240A168A150317C701E330C6000A121A
:103030000313A2270A168316E101A030E000E33053
:1030400084008313003000040319402883120317FF
:103050009C0104089B001C10831B1C140008CA0060
:103060000A128A110313A2250A168A1503171B08D0
:10307000840083131C188317840A831603132228E1
:10308000831203179C01A0309B008A11031339227D
:103090008A150A12C6270A168A150A164E2E831694
:1030A000DF08031DD328DE08031DD328DD08031D18
:1030B000D3285C08043C031CD3280A1283129327EC
:1030C0000A16013083165C07831203179B008316D0
:1030D00003135D08831203179C00003003180130AE
:1030E0009C07831603135E08831203179D000030AC
:1030F000031801309D07831603135F08831203171B
:103100009E000030031801309E07031313080317B5
:103110001B08031393008316141C8C28323083126F
:103120000317CD000A128A110313CC240A168A153C
:103130000317C701E330C6000A120313A2270A16B9
:103140008316E101A030E000E330840083130030F7
:1031500000040319C528831203179C0104089B006F
:103160001C10831B1C140008CA000A128A110313C6
:10317000A2250A168A1503171B08840083131C183E
:103180008317840A83160313A728831203179C014D
:10319000A0309B008A11031339228A150A12C62710
:1031A0000A16DC28831683126C1403179C019B01FA
:1031B0008A11031339228A158A150A165E2E831680
:1031C000E101A030E0001030840083126008031792
:1031D000B30003135F080317B2000A128A11031326
:1031E00049270A168A1503179C01A0309B008A11F3
:1031F000031339228A158A150A166E2E8316E101E9
:10320000A030E00010308400831262080317B3007E
:10321000031361080317B2000A128A110313492726
:103220000A168A1503179C01A0309B008A1103130C
:1032300039228A158A150A167E2E8316E101A030DE
:10324000E00010308400831264080317B3000313F6
:1032500063080317B2000A128A11031349270A16DA
:103260008A1503179C01A0309B008A110313392291
:103270008A158A150A168E2E00306718013003173A
:103280009B0083160313E101A030E00083120317B3
:103290001B08C6001B30C7000A1203136E210A1652
:1032A00003179C01A0309B008A11031339228A1551
:1032B0008A150A169E2E8316E101A030E0008312C3
:1032C00003179B011B080A128A1103133E200A16DA
:1032D0008A1500380319782903179B0ACA000A12B5
:1032E0008A110313A2250A168A15031762290313EC
:1032F00003179C01A0309B008A11031339228A1501
:103300008A150A16C02E8316DF08031D912ADE08CF
:10331000031D912A5D08273C031C912A031D942953
:103320005C08103C031C912A0A12831293270A1688
:1033300013083C3093008316141C9C290130E100D3
:103340001030E000413084005F0883120317B6009C
:10335000831603135E0883120317B5008316031345
:103360005D0883120317B400831603135C088312ED
:103370000317B3000A128A110313B5250A168A151A
:1033800020300317CA000A128A110313A2250A1655
:103390008A1501300317B3001030B2000A128A11E7
:1033A000031319260A168A1532300317CD000A12A4
:1033B0008A110313CC240A168A150317C701E330B8
:1033C000C6000A120313A2270A160317B301E3303B
:1033D000B2000A12031300200A167A0803179E008F
:1033E00079089D0078089C0077089B0083160313DA
:1033F0005C08831203171B02031D602A8316031344
:103400005D08831203171C02031D602A8316031331
:103410005E08831203171D02031D602A831603131F
:103420005F08831203171E02031D602A831603130D
:103430005D088312E00083165C088312DF00031727
:10344000B201031360080317B40003135F080317E6
:10345000B3000A128A1103133E220A168A150317B3
:10346000B2010A128A1103130B220A168A1579086F
:10347000FA0078085F02031D412A7A0860020319E6
:10348000422A67158316E101A030E0001030840065
:10349000831260080317B30003135F080317B20019
:1034A0000A128A11031349270A168A1503179C0169
:1034B000A0309B008A11031339228A158C2A031726
:1034C0000313EC158316E101A030E00041308400C5
:1034D0005F0883120317B600831603135E08831276
:1034E0000317B500831603135D0883120317B40096
:1034F000831603135C0883120317B3000A128A11A0
:103500000313B5250A168A1503179C01A0309B00EA
:103510008A11031339228A150A12C6270A16BD2AF0
:10352000831683126C148316E101A030E000413051
:1035300084005F0883120317B600831603135E0826
:1035400083120317B500831603135D088312031754
:10355000B400831603135C0883120317B3000A1226
:103560008A110313B5250A168A1503179C01A0308A
:103570009B008A11031339228A158A150A16D02E48
:103580008316DF08031DD02BDE08031DD02B5D083A
:10359000273C031CD02B031DD12A5C08103C031CC4
:1035A000D02B0A12831293270A1613083D3093007A
:1035B0008316141CD92A0130E1001030E00041309C
:1035C00084005F0883120317B600831603135E0896
:1035D00083120317B500831603135D0883120317C4
:1035E000B400831603135C0883120317B3000A1296
:1035F0008A110313B5250A168A1520300317CA004D
:103600000A128A110313A2250A168A15013003171C
:10361000B3001030B2000A128A11031319260A16D9
:103620008A1532300317CD000A128A110313CC24F5
:103630000A168A150317C701E330C6000A120313DE
:10364000A2270A160317B301E330B2000A120313CC
:1036500000200A167A0803179E0079089D00780852
:103660009C0077089B00831603135C0883120317E2
:103670001B02031D9F2B831603135D088312031780
:103680001C02031D9F2B831603135E08831203176E
:103690001D02031D9F2B831603135F08831203175C
:1036A0001E02031D9F2B831603135D088312E20085
:1036B00083165C088312E10002300317B200031383
:1036C00062080317B400031361080317B3000A125A
:1036D0008A1103133E220A168A1502300317B2001C
:1036E0000A128A1103130B220A168A157908FA00A6
:1036F00078086102031D802B7A0862020319812B6E
:1037000067158316E101A030E000103084008312B9
:1037100062080317B300031361080317B2000A120B
:103720008A11031349270A168A1503179C01A03032
:103730009B008A11031339228A15CB2B031703131D
:10374000EC158316E101A030E000413084005F08F1
:1037500083120317B600831603135E088312031740
:10376000B500831603135D0883120317B400831694
:1037700003135C0883120317B3000A128A110313A0
:10378000B5250A168A1503179C01A0309B008A11E3
:10379000031339228A150A12C6270A16FC2B831630
:1037A00083126C148316E101A030E00041308400E4
:1037B0005F0883120317B600831603135E08831293
:1037C0000317B500831603135D0883120317B400B3
:1037D000831603135C0883120317B3000A128A11BD
:1037E0000313B5250A168A1503179C01A0309B0008
:1037F0008A11031339228A158A150A16E02E8316B8
:10380000DF08031D0F2DDE08031D0F2D5D08273C6B
:10381000031C0F2D031D102C5C08103C031C0F2DE6
:103820000A12831293270A1613083E309300831658
:10383000141C182C0130E1001030E00041308400ED
:103840005F0883120317B600831603135E08831202
:103850000317B500831603135D0883120317B40022
:10386000831603135C0883120317B3000A128A112C
:103870000313B5250A168A1520300317CA000A1249
:103880008A110313A2250A168A1501300317B30003
:103890001030B2000A128A11031319260A168A156B
:1038A00032300317CD000A128A110313CC240A16F2
:1038B0008A150317C701E330C6000A120313A227B3
:1038C0000A160317B301E330B2000A1203130020F3
:1038D0000A167A0803179E0079089D0078089C0054
:1038E00077089B00831603135C08831203171B02DF
:1038F000031DDE2C831603135D08831203171C02BD
:10390000031DDE2C831603135E08831203171D02AA
:10391000031DDE2C831603135F08831203171E0298
:10392000031DDE2C831603135D088312E400831647
:103930005C088312E30004300317B2000313640829
:103940000317B400031363080317B3000A128A11A4
:1039500003133E220A168A1504300317B2000A1216
:103960008A1103130B220A168A157908FA007808BF
:103970006302031DBF2C7A0864020319C02C67156B
:103980008316E101A030E000103084008312640847
:103990000317B300031363080317B2000A128A1156
:1039A000031349270A168A1503179C01A0309B00B0
:1039B0008A11031339228A150A2D03170313EC15F4
:1039C0008316E101A030E000413084005F088312DB
:1039D0000317B600831603135E0883120317B5009E
:1039E000831603135D0883120317B40083160313B1
:1039F0005C0883120317B3000A128A110313B5255A
:103A00000A168A1503179C01A0309B008A11031324
:103A100039228A150A12C6270A163B2D83168312ED
:103A20006C148316E101A030E000413084005F088F
:103A300083120317B600831603135E08831203175D
:103A4000B500831603135D0883120317B4008316B1
:103A500003135C0883120317B3000A128A110313BD
:103A6000B5250A168A1503179C01A0309B008A1100
:103A7000031339228A158A150A16F02E8316E101DE
:103A8000A030E000831203179B011B080A128A1161
:103A900003135E200A168A1503179B0AF700CA0053
:103AA0000A128A110313A2250A168A150D3003176C
:103AB0001B02031D452D9C01A0309B000A1203131D
:103AC00050260A168316DF08031D962DDE08031DF7
:103AD000962DDD08031D962D5C08633C031C962D76
:103AE0005C088312E50005300317B200B40103132C
:103AF00065080317B3000A128A1103133E220A163F
:103B00008A1505300317B2000A128A1103130B221B
:103B10000A168A157908FA0078086502031D932DA4
:103B2000FA080319942D6715982D831683126C14C7
:103B30008316E101A030E000413084005F08831269
:103B40000317B600831603135E0883120317B5002C
:103B5000831603135D0883120317B400831603133F
:103B60005C0883120317B3000A128A110313B525E8
:103B70000A168A1503179C01A0309B008A110313B3
:103B800039228A158A150A16002F8A1100288A15EB
:103B9000640003179B010A120313752E0A16F80816
:103BA00003190A2FEC1603179C01CC309B009E01D1
:103BB0002F309D000A1203134C270A16F808031D24
:103BC000E52D8A11AC2D8A150A2F03179C01CC30E4
:103BD0009B009E0131309D000A1203134C270A16E8
:103BE000F808031DF72D8A11642E8A150A2F031772
:103BF0009C01CC309B009E0133309D000A120313C0
:103C00004C270A16F808031D092E8A11F32E8A156F
:103C10000A2F03179C01CC309B009E0136309D007B
:103C20000A1203134C270A16F808031D1B2E8A11CB
:103C30001B2F8A150A2F03179C01CC309B009E0175
:103C400039309D000A1203134C270A16F808031D89
:103C50002D2E8A11582F8A150A2F03179C01CC305C
:103C60009B009E013C309D000A1203134C270A164C
:103C7000F808031D3F2E8A11A72F8A150A2F031754
:103C80009C01CC309B009E013F309D000A12031323
:103C90004C270A16F808031D4F2E00280A2F031779
:103CA0009C01CC309B009E0142309D000A12031300
:103CB0004C270A16F808031D5F2E4F280A2F0317FA
:103CC0009C01CC309B009E0145309D000A120313DD
:103CD0004C270A16F808031D6F2EDF280A2F03173A
:103CE0009C01CC309B009E0148309D000A120313BA
:103CF0004C270A16F808031D7F2EFE280A2F0317EB
:103D00009C01CC309B009E014B309D000A12031396
:103D10004C270A16F808031D8F2E1D290A2F03179A
:103D20009C01CC309B009E014E309D000A12031373
:103D30004C270A16F808031D9F2E3C290A2F03174B
:103D40009C01CC309B009E0151309D000A12031350
:103D50004C270A16F808031DB12E8A11EB2F8A157D
:103D60000A2F03179C01CC309B009E0154309D000C
:103D70000A1203134C270A16F808031DC12E5B29EB
:103D80000A2F03179C01CC309B009E0157309D00E9
:103D90000A1203134C270A16F808031DD12E832993
:103DA0000A2F03179C01CC309B009E0159309D00C7
:103DB0000A1203134C270A16F808031DE12EC02A25
:103DC0000A2F03179C01CC309B009E015B309D00A5
:103DD0000A1203134C270A16F808031DF12EFF2BB5
:103DE0000A2F03179C01CC309B009E015D309D0083
:103DF0000A1203134C270A16F808031D012F3E2D43
:103E00000A2FE71703179C019B018A11031339221C
:103E10008A15EC12C82D8A150A16D92F840183132E
:103E20001F308305193083169900A6309800903012
:103E30008312980083161F149F141F159F110730BB
:103E40009C008312A901AA014C30AF00B00143309D
:103E5000B100B2015330B3004530B400B5013F307A
:103E6000B6005630B700B8013F30B9007630BA001E
:103E7000BB013F30BC004930BD00BE013F30BF0038
:103E80006930C000C1013F30C2006730C300C401C7
:103E90003F30C5004F30C600C7013F30C8006F300B
:103EA000C900CA013F30CB005430CC00CD013F30B7
:103EB000CE004330CF00D0013F30D1005330D2008C
:103EC000D3013F30D4007330D500D6014F30D70036
:103ED000D8016F30D900DA015430DB00DC015330F7
:103EE000DD00DE01DF01E001E101E201E301E401C7
:103EF000E501E6016710E801E901EA01EB01E710DD
:103F00006711E7116712E7126713E7136C10EC10E3
:103F10006C11EC11F101F201F301F401ED01EE017C
:103F2000F501F6010330EF00FC016C16EC126C1386
:103F3000EC137D10FD107D110130FE008316BE01D3
:103F4000DA01DB01DC01DD01DE01DF01FD117D12A3
:103F5000FD127D13E001E101FF30E2000308183992
:103F6000F7000E08033977040E148E148315031618
:103F7000033A83120319C32F083A0319C32F133AC4
:103F80000319C52FC72F6C17C72F6C13C72F0A1221
:103F90008A11E9290A168A158316621462088700B5
:103FA0008312071CD82F6C120A12B7290A16D92FB0
:0A3FB000C52D0A12F52F0A16DC2FAA
:02400E00313748
:00000001FF
